:10000000B1EF08F000000000000000000000000058
:1000100000000000000000000000000000000000E0
:10002000000000008005A5050000000000000000A1
:1000300000000000000000000000000000000F04AD
:10004000000000000000FD030000000000000000B0
:1000500000000000000000000000000000000000A0
:100060000000000000000000000000000000000090
:100070000000000000000000000000000000000080
:100080000000000000000000000000000000000070
:100090000000000000000000000000000000000060
:0C00A00000000000000000000000000054
:0C00AC00000E3D01E1BF010E006E1200CD
:0C00B800000E3D01F9BF010E006E1200A9
:0400C400F3DF120054
:0400C800F7DF12004C
:1000CC00FBDF005202E10000FBD760005FF6D2FDBF
:0200DC00120010
:1000DE00F4DF005202E10000FBD760005FF6EAFD9C
:0200EE001200FE
:0800F00096C197F1EBDF12004D
:0800F80096C197F1F0DF120040
:0E010000550E3A01BF6FAA0EBF6FBF911200DD
:08010E0096C197F1E5DF120034
:0801160096C197F1D8DF120039
:0E011E00550E3A01BF6FAA0EBF6FBF811200CF
:10012C00D250026ED29E0500FF6A0150FE6E005046
:08013C00FD6E02BED28E12001E
:1001440001019251170802E2006A0ED39351000A8A
:10015400D8A4B1D0955301E0D1DF60D0600053F64C
:1001640000FAA5D0600053F601FAA1D0600053F65E
:1001740002FA9DD0600053F603FA99D0600053F65A
:1001840004FA95D0600053F605FA91D0600053F656
:1001940006FA8DD0600053F607FA89D0600053F652
:1001A40008FA85D0600053F609FA81D0600053F64E
:1001B4000AFA7DD0600053F60BFA79D0600053F64A
:1001C4000CFA75D0600053F60DFA71D0600053F646
:1001D4000EFA6DD0600053F60FFA69D0600053F642
:1001E40010FA65D0600053F611FA61D0600053F63E
:1001F40012FA5DD0600053F613FA59D0600053F63A
:1002040014FA55D0600053F615FA51D0600053F635
:1002140016FA4DD0600053F617FA49D001019251F5
:10022400000A9CE09251010A9DE09251020A9EE06C
:100234009251030A9FE09251040AA0E09251050AE8
:10024400A1E09251060AA2E09251070AA3E092515A
:10025400080AA4E09251090AA5E092510A0AA6E00C
:1002640092510B0AA7E092510C0AA8E092510D0A90
:10027400A9E092510E0AAAE092510F0AABE0925102
:10028400100AACE09251110AADE09251120AAEE0AC
:100294009251130AAFE09251140AB0E09251150A38
:1002A400B1E09251160AB2E09251170AB3E001018B
:1002B400955301E032DF01019351010AD8A451D1D1
:1002C400955301E01BDFA4D060004BF6C0FA45D182
:1002D40060004BF6C1FA41D160004BF6C2FA3DD141
:1002E40060004BF6C3FA39D160004BF6C4FA35D13D
:1002F40060004BF6C5FA31D160004BF6C6FA2DD139
:1003040060004BF6C7FA29D160004BF6C8FA25D134
:1003140060004BF6C9FA21D160004BF6CAFA1DD130
:1003240060004BF6CBFA19D160004BF6CCFA15D12C
:1003340060004BF6CDFA11D160004BF6CEFA0DD128
:1003440060004BF6CFFA09D160004BF6D0FA05D124
:1003540060004BF6D1FA01D160004BF6D2FAFDD021
:1003640060004BF6D3FAF9D060004BF6D4FAF5D01E
:1003740060004BF6D5FAF1D060004BF6D6FAEDD01A
:1003840060004BF6D7FAE9D060004BF6D8FAE5D016
:1003940060004BF6D9FAE1D060004BF6DAFADDD012
:1003A40060004BF6DBFAD9D060004BF6DCFAD5D00E
:1003B40060004BF6DDFAD1D060004BF6DEFACDD00A
:1003C40060004BF6DFFAC9D060004BF6E0FAC5D006
:1003D40060004BF6E1FAC1D060004BF6E2FABDD002
:1003E40060004BF6E3FAB9D060004BF6E4FAB5D0FE
:1003F40060004BF6E5FAB1D060004BF6E6FAADD0FA
:1004040060004BF6E8FAA9D060004BF6E9FAA5D0F3
:1004140001019451000AD8B457D79451010AD8B4B1
:1004240057D79451020AD8B457D79451030AD8B471
:1004340057D79451040AD8B457D79451050AD8B45D
:1004440057D79451060AD8B457D79451070AD8B449
:1004540057D79451080AD8B457D79451090AD8B435
:1004640057D794510A0AD8B457D794510B0AD8B421
:1004740057D794510C0AD8B457D794510D0AD8B40D
:1004840057D794510E0AD8B457D794510F0AD8B4F9
:1004940057D79451100AD8B457D79451110AD8B4E5
:1004A40057D79451120AD8B457D79451130AD8B4D1
:1004B40057D79451140AD8B457D79451150AD8B4BD
:1004C40057D79451160AD8B457D79451170AD8B4A9
:1004D40057D79451180AD8B457D79451190AD8B495
:1004E40057D794511A0AD8B457D794511B0AD8B481
:1004F40057D794511C0AD8B457D794511D0AD8B46D
:1005040057D794511E0AD8B457D794511F0AD8B458
:1005140057D79451200AD8B457D79451210AD8B444
:1005240057D79451220AD8B457D79451230AD8B430
:1005340057D79451240AD8B457D79451250AD8B41C
:1005440057D79451260AD8B457D79451270AD8B408
:1005540057D79451280AD8B457D70101955301E0CD
:10056400DCDDA8D0010193B102D0C29001D0C280D9
:10057400F9D0010193B102D0C29201D0C282F2D06B
:10058400010193B102D0C29401D0C284EBD0010125
:1005940093B102D0C29601D0C286E4D0010193B1D6
:1005A40002D0C29801D0C288DDD0010193B102D03B
:1005B400C29A01D0C28AD6D0010193B102D0C29CA2
:1005C40001D0C28CCFD0010193B102D0C29E01D020
:1005D400C28EC8D0010193B102D0C39001D0C380B0
:1005E400C1D0010193B102D0C39201D0C382BAD069
:1005F400010193B102D0C39401D0C384B3D00101EB
:1006040093B102D0C39601D0C386ACD0010193B19B
:1006140002D0C39801D0C388A5D0010193B102D000
:10062400C39A01D0C38A9ED0010193B102D0C39C66
:1006340001D0C38C97D0010193B102D0C39E01D0E5
:10064400C38E90D0010193B102D0C49001D0C48074
:1006540089D0010193B102D0C49201D0C48282D066
:10066400010193B102D0C49401D0C4847BD00101B0
:1006740093B102D0C49601D0C48674D0010193B161
:1006840002D0C49801D0C4886DD0010193B102D0C6
:10069400C49A01D0C48A66D0010193B102D0C49C2B
:1006A40001D0C48C5FD0010193B102D0C49E01D0AB
:1006B400C48E58D001019251000AD8B453D7925134
:1006C400010AD8B456D79251020AD8B459D79251D4
:1006D400030AD8B45CD79251040AD8B45FD79251B4
:1006E400050AD8B462D79251060AD8B465D7925194
:1006F400070AD8B468D79251080AD8B46BD7925174
:10070400090AD8B46ED792510A0AD8B471D7925153
:100714000B0AD8B474D792510C0AD8B477D7925133
:100724000D0AD8B47AD792510E0AD8B47DD7925113
:100734000F0A81E09251100A85E09251110A89E072
:100744009251120A8DE09251130A91E09251140AC7
:1007540095E09251150A99E09251160A9DE0925142
:0A076400170AA1E0FF0E006E12005C
:10076E00600097F5E1FF60009BF5E2FF60003FF649
:0E077E00E6FF63C100F064C101F0D1DC12009F
:10078C008FC192F190C193F191C194F1010E0101CD
:06079C00956FD2DC120093
:1007A200160E01018F6F906B130E916FEEDF170E15
:1007B20001018F6F010E906F250E916FE6DF12001F
:1007C2000B6A0A6A096A086A0E6A03340836045018
:1007D200085E0550D8A0053C095E0650D8A0063C2C
:1007E2000A5E0750D8A0073C0B5EE86AD8A0010E4B
:1007F2000E5E0336070E0C6E0334083609360A36CF
:100802000B360E36045003A012D0085E0550D8A055
:10081200053C095E0650D8A0063C0A5E0750D8A0E7
:10082200073C0B5EE86AD8A0010E0E5E11D00826C6
:100832000550D8B0053C09260650D8B0063C0A2619
:100842000750D8B0073C0B26E86AD8B0010E0E2636
:1008520003360C2ED1D70234083609360A360B3647
:100862000E36045003A012D0085E0550D8A0053CF5
:10087200095E0650D8A0063C0A5E0750D8A0073C85
:100882000B5EE86AD8A0010E0E5E11D00826055054
:10089200D8B0053C09260650D8B0063C0A260750B7
:1008A200D8B0073C0B26E86AD8B0010E0E260236F5
:1008B200070E0C6E0234083609360A360B360E362F
:1008C200045002A012D0085E0550D8A0053C095E73
:1008D2000650D8A0063C0A5E0750D8A0073C0B5E23
:1008E200E86AD8A0010E0E5E11D008260550D8B0D5
:1008F200053C09260650D8B0063C0A260750D8B057
:10090200073C0B26E86AD8B0010E0E2602360C2EE2
:10091200D1D70134083609360A360B360E36045062
:1009220002A012D0085E0550D8A0053C095E065010
:10093200D8A0063C0A5E0750D8A0073C0B5EE86AC6
:10094200D8A0010E0E5E11D008260550D8B0053C85
:1009520009260650D8B0063C0A260750D8B0073CF4
:100962000B26E86AD8B0010E0E260136070E0C6E71
:100972000134083609360A360B360E36045001A009
:1009820012D0085E0550D8A0053C095E0650D8A0DA
:10099200063C0A5E0750D8A0073C0B5EE86AD8A066
:1009A200010E0E5E11D008260550D8B0053C09266E
:1009B2000650D8B0063C0A260750D8B0073C0B2692
:1009C200E86AD8B0010E0E2601360C2ED1D70034BB
:1009D200083609360A360B360E36045001A012D0FC
:1009E200085E0550D8A0053C095E0650D8A0063C1A
:1009F2000A5E0750D8A0073C0B5EE86AD8A0010E39
:100A02000E5E11D008260550D8B0053C09260650C6
:100A1200D8B0063C0A260750D8B0073C0B26E86A35
:100A2200D8B0010E0E260036070E0C6E00340836C2
:100A320009360A360B360E36045000A012D0085E74
:100A42000550D8A0053C095E0650D8A0063C0A5EB7
:100A52000750D8A0073C0B5EE86AD8A0010E0E5ED4
:100A620011D008260550D8B0053C09260650D8B04A
:100A7200063C0A260750D8B0073C0B26E86AD8B0D5
:100A8200010E0E2600360C2ED1D700B00ED0045027
:100A920008260550D8B0053C09260650D8B0063CB9
:0C0AA2000A260750D8B0073C0B261200B3
:0C0AAE006F00A0F701F001C000F0120082
:100ABA0001017F510308D8A07F6B80510308D8A099
:100ACA00806BF00E3D01F21701017F513D01F213D7
:100ADA00300EF21380C100F000360090003600900C
:100AEA0000360090003600900050F413F38F120085
:100AFA000101826B6000FFF5E9FF600003F6EAFF7F
:100B0A006F00B8FF81F18151000A0FE081C18FF1B6
:100B1A0029DE0101822B82517F25E96E000E802198
:0C0B2A00EA6E6F00B8FF81F1EED71200F8
:100B36007FC167F180C168F181C169F182C16AF143
:100B460083C163F184C164F185C165F186C166F133
:100B560087C171F188C172F189C173F18AC174F1DB
:100B66008BC16DF18CC16EF18DC16FF18EC170F1CB
:020B760012006B
:100B7800086A096A100E0C6E0134083609360450EA
:100B8800085E0550D8A0053C095ED8B007D00450CF
:100B980008260550D8B0053C0926D89000360136FD
:060BA8000C2EEAD712003A
:100BAE000001B76BB86B000EB85D02E14F0EB75D7A
:100BBE0018E20D0EB725E16E010EB821E26E6F0040
:100BCE0087FFE1FF6F008BFFE2FFE66A010EB7259C
:100BDE00006E000EB821016E00C0B7F001C0B8F073
:100BEE00E2D701010D6B0001B76BB86B01015D6BB4
:100BFE005E6B5F6B606B0B6B0C6B3D01F289F96B7F
:100C0E00FA6B390193876F00A0F75FF05F6A1200ED
:100C1E00C1DD500E01017F6F0D0E806F000E816FD2
:100C2E00000E826FF80E836F000E846F960E856F26
:100C3E00010E866FFF0E876FFF0E886F000E896F95
:100C4E00000E8A6FC80E8B6F000E8C6F000E8D6FAC
:0E0C5E00000E8E6F69DF7F6B806B28DF120047
:100C6C0001017B6B7C6B000E7C5D02E10A0E7B5DEF
:100C7C000BE27B517925E16E7C517A21E26E200EDC
:100C8C00E66E7B4B7C2BEFD77B517925E16E7C514B
:100C9C007A21E26EE66A010E7B5F000E7C5B7B5173
:100CAC0079257D6F7C517A217E6F0A0E046E000EC1
:100CBC00056E066E076E75C100F076C101F077C146
:100CCC0002F078C103F077DD08C000F009C001F034
:100CDC000AC002F00BC003F0300E00266000F7F5DE
:100CEC00E1FF6000FBF5E2FF600003F0E6FF0A0E97
:100CFC00046E000E056E066E076E75C100F076C1AF
:100D0C0001F077C102F078C103F055DD00C075F138
:100D1C0001C076F102C077F103C078F1000E046EC9
:100D2C00031808E10450021805E10450011802E10F
:100D3C000050000A01E105D0010E7B5F000E7C5BC8
:040D4C00AED712000C
:040D5000AEDE120001
:100D54003901C06BC16BC26BFF0ECA6E010E3A0142
:100D6400406F830EC26E41934293C298BA88C29672
:100D7400BA86C29ABA9A506BCB6AFF0EC36EFF0E44
:100D8400516F3E01BC6BB86BCC6AB30EC46E3A01B2
:100D9400606B80EC00F0130E166F170EE56F150EE6
:100DA400E66F100ED16F110ED26F8FEC00F03E0182
:0A0DB400C16BC19FC183C191120001
:100DBE0009006F00D7FFE6FF0006FAE10106F8E131
:020DCE00120011
:100DD00075C100F00032009E0032009E0032009E7D
:100DE0000032009E4C0E0024F66E190EF76E000EB7
:100DF000F722000EF86E000EF82209006F00D4FFF3
:100E000000F06000DBF5E1FF6000DFF5E2FF60006D
:100E100003F0E6FF010E01017625E16E000E772159
:100E2000E26E0F0E7515006E4C0E0024F66E190E54
:100E3000F76E000EF722000EF86E000EF822090081
:100E40006F00D4FF00F0600003F0E6FF020E76258D
:0C0E5000E16E000E7721E26EE66A1200EF
:100E5C000101796B050E795D0AE279517725E16E16
:100E6C00000E7821E26E200EE66E792BF3D77951C5
:100E7C007725E16E000E7821E26EE66A79077951EA
:100E8C0077257A6F000E78217B6F0A0E046E000EA8
:100E9C00056E75C100F076C101F068DE08C000F087
:100EAC0009C001F0300E00266000EBF5E1FF600098
:100EBC00EFF5E2FF600003F0E6FF0A0E046E000E91
:100ECC00056E75C100F076C101F050DE00C075F101
:100EDC0001C076F1000E011802E1000E001801E1CC
:080EEC0002D07907CCD71200F7
:0C0EF40075C17FF176C180F1FEDD1200B7
:100F00000D0E0101966F7CEC00F00A0E0101966F48
:060F10007CEC00F0120071
:100F160075C104F076C105F004C002F005C003F007
:100F2600044A052A77C100F078C101F00101774B28
:100F3600782B600003F0E9FF600007F0EAFF60002D
:100F46000BF0E1FF60000FF0E2FF6F00BBFFE6FF72
:100F560060000BF0E9FF60000FF0EAFFEE5201E0DF
:0C0F6600DBD775C100F076C101F012006D
:100F72006000D7F5F6FF6000DBF5F7FF6000DFF5F4
:100F8200F8FF09006F00D4FF01F00150000816E2DB
:100F92006000D7F5F6FF6000DBF5F7FF6000DFF5D4
:100FA200F8FF09006F00D4FF96F17CEC00F0010E0F
:0E0FB20001017527000E76237723DAD712008F
:100FF40000C020F06F0084FF21F06F0088FF22F012
:10100400300E55243D01EA6F554A562A000E006EF3
:101014005650005C02E15550090802E20001608567
:10102400BA863901A39F20C000F0600087F0E1FF79
:0810340060008BF0E2FF1100E7
:10103C0000C01DF001C01CF06F0084FF1EF06F009B
:10104C0088FF1FF07FDE00C05FF03D01F9AB0FD0D1
:10105C00F99B010E01016B25006E000E6C21016ED7
:10106C0000C06BF101C06CF16F00A0F75FF03D01A7
:10107C00F9A70ED0010E01016B25006E000E6C213C
:10108C00016E00C06BF101C06CF15CDE00C05FF062
:10109C005F500D0A0AE05F500A0A07E06051000831
:1010AC0002E15F514F0801E32AD00101010E0B6FE1
:1010BC00000E0C6F0D0E0001B725E16E010EB8216C
:1010CC00E26E6F0087FFE1FF6F008BFFE2FFE66AC5
:1010DC0039019397B7C05FF1B8C060F10001B76BED
:1010EC00B86B01016051000802E15F514F0804E246
:1010FC00020E0B6F000E0C6F3901949521D001017B
:10110C000B6B0C6B0D0E0001B725E16E010EB821B7
:10111C00E26E6F0087FFE1FF6F008BFFE2FF600064
:10112C007FF1E6FFB7C05FF1B8C060F1010EB725E3
:10113C00006E000EB821016E00C0B7F001C0B8F00F
:10114C001DC000F01CC001F060007BF0E1FF6000EE
:06115C007FF0E2FF11002C
:10116200B8EC0CF0600E3901D96F080EDF6FDE6B40
:10117200D76AD66A080ED56EECDD0101616B626B2F
:10118200800E6219006E800E005C02E1500E615DFD
:1011920010E2670E6125E16E000E6221E26E6F00C1
:1011A20087FFE1FF6F008BFFE2FFE66A614B622B74
:1011B200E7D7616B626B800E6219006E800E005C75
:1011C20002E1500E615D10E2BB0E6125E16E000E80
:1011D2006221E26E6F0087FFE1FF6F008BFFE2FF8B
:1011E200E66A614B622BE7D70001B76BB86B01016E
:1011F2005F6B606BBB0E0001656F000E666F400E89
:101202003D01F56F030EF66FF28F08DD500E0101FE
:101212007F6F0D0E806F000E816F000E826FF80ED1
:10122200836F000E846F960E856F010E866FFF0E20
:10123200876FFF0E886F000E896F000E8A6FC80ECF
:101242008B6F000E8C6F000E8D6F000E8E6F72DC36
:10125200110E0B6E3C0E0C6ECB0E0D6E0D2EFED7CC
:101262000C2EFCD70B2EFAD70C0E966F7CEC00F0EE
:1012720046DE290E0101756F190E766F000E776F2B
:1012820077DEE20E0101756F180E766F000E776F32
:101292006FDECC0E0101756F170E766F000E776F41
:1012A20067DE1C0E0101756F180E766F000E776FE8
:1012B2005FDE790E0101756F170E766F000E776F84
:1012C20057DEB20E0101756F150E766F000E776F45
:1012D2004FDE3B0E0101756F190E766F000E776FB0
:1012E20047DEFC0E0101756F180E766F000E776FE8
:1012F2003FDE220E0101756F170E766F000E776FBB
:1013020037DE65C075F166C076F1230E0101776F95
:10131200000E786FFFDD65C075F166C076F1E9DD1C
:101322000D0E966F7CEC00F0290E0B6E960E0C6E75
:101332007F0E0D6E0D2EFED70C2EFCD70B2EFAD77C
:10134200000E0001B96FFA0EBA6FC70E0101756F78
:10135200180E766F000E776F0BDEB9C075F1BAC04A
:1013620076F1670E0101776F000E786F76DD670EFA
:10137200756F000E766FBDDDC2DD6B0E0101756FFC
:10138200180E766F000E776FF3DD010E3F01216FAD
:10139200236B226B126B136B146B156B166B176B33
:1013A200186B196B1A6B1E8F1E991E971E951E9332
:1013B2001E911E9B1F6B1F9F1F9D0A0E1F13140E53
:1013C2000101756F190E766F000E776FD1DD590E20
:1013D2005D6E000E5E6EFF0E596E7F0E5A6E000E2F
:1013E2005B6E5C6E020E5D24E96E000E5E20EA6E9C
:1013F2006F00A7FFE9FF6F00ABFFEAFF6F00B8FFC6
:1014020075F1670E0101766F000E776FE0DC670EF3
:10141200756F000E766F6DDD010E5D24E96E000EB4
:101422005E20EA6E6F00A7FFE9FF6F00ABFFEAFFE5
:101432006F00B8FF75F1670E766F000E776FC7DC2D
:10144200670E756F000E766F54DD600077F1E9FF6D
:1014520060007BF1EAFF6F00B8FF75F1670E766FEF
:10146200000E776FB4DC670E756F000E766F41DD8C
:1014720046DD596A5A6A5B6A5C6A610E576E000EF3
:10148200586E0001616B626B636B646BB80E010195
:10149200756F160E766F000E776F6ADD3901A19DAA
:1014A200918D818DA19B919BA19F918F818FAC0E7C
:1014B2000101756F180E766F000E776F59DD3D01D1
:1014C200F86B800EF46F3901818BA18B3D01FA6BB1
:1014D200390193878387D28EBA98596A5A6A5B6AAE
:1014E2005C6A0001616B626B636B646BBA983F016B
:1014F2001E8F1F8F520E0B6E400E0C6EC70E0D6E9E
:101502000D2EFED70C2EFCD70B2EFAD700000000B2
:10151200BA885C50000808E15B50000805E15A50A7
:10152200000802E1595000081EE259C075F15AC084
:1015320076F15BC077F15CC078F1670E0101796FDB
:10154200000E7A6F36EC06F0680E756F190E766F24
:10155200000E776F0DDD670E0101756F000E766F5D
:10156200C8DCCDDC08D0FC0E0101756F150E766F5C
:10157200000E776FFDDCD7EC05F0000E01010C19AF
:1015820002E1010E0B1912E1BA985C0E756F190E89
:10159200766F000E776FECDC0D0E0101756F010E98
:1015A200766FA7DCACDC01015D6B5E6B95D7FFD774
:101600006F0084FF18F06F0088FF19F02A0E3D016B
:10161000EA6F3901A19D600077F1E1FF60007BF185
:10162000E2FF6F0057FCE6FF010E5D24E16E000E45
:101630005E20E26E6F0087FFE1FF6F008BFFE2FF2D
:101640006F005BFCE6FF020E5D24E16E000E5E2083
:10165000E26E6F0087FFE1FF6F008BFFE2FF6F001C
:101660005FFCE6FF030E5D24E16E000E5E20E26E7D
:101670006F0087FFE1FF6F008BFFE2FFE66A3F012B
:101680001F9F1E9F600063F0E1FF600067F0E2FFB4
:02169000110047
:101694006F0084FF1AF06F0088FF1BF0240E3D01D9
:1016A400EA6F3901A19F60006BF0E1FF60006FF009
:0416B400E2FF110040
:1019700010EE23F0340E006E010E016EC00EF66EF6
:0E1980000F0EF76E000EF86EDFEC06F0120090
:100FC00020436865636B205265676C616765204FDD
:100FD000534354554E452C20617665632046726517
:100FE000716D657465722073757220524136200DE3
:020FF0000A00F5
:020FF2000000FD
:1015B20020434F4E464947203A2050313846323771
:1015C2004B34325F466F73635F696E7465726E652A
:1015D2005F776974685F504C4C5F36344D487A5F70
:1015E200776974685F566563746F7265645F4954A6
:0A15F2002E6366677363680D0A003C
:0215FC002E00BF
:1016B800205465737420534D543120656E206D6F2E
:1016C8006465203130203A206D6F646520313031F7
:1016D80030204649475552452032352D32323A207E
:1016E80057494E444F57454420434F554E54455251
:1016F800204D4F44452053494E474C4520414351C6
:101708005549534954494F4E2054494D494E472055
:0A1718004449414752414D0D0A00BB
:10172200204841524457415245203A0D0A20205345
:101732004D543157494E203D20524330203D2042E6
:101742006173652064652074656D70732031736503
:10175200632020202020534D54315349473D2052CD
:1017620043313D207369676E616C20E0206D6573C3
:07177200757265720D0A009B
:1017790020536F75726365203A20426173655F314A
:10178900384632374B34325F466F73635F696E7424
:1017990065726E655F36344D687A5F5541525431D2
:1017A9005F534D545F467265716D657465725F5420
:1017B9006573745F5F323032312D313131302E63D0
:0317C9000D0A0006
:1017CC00204469726563746F7279203A20433A5CE5
:1017DC005F4D696B726F435C5F4D657350726F6ADE
:1017EC006574735F4D696B726F435C5F3138463261
:1017FC00374B34325F546573745F534D54315F32E1
:10180C0034626974735F636F756E7465720D0A0070
:10181C002050726F6A6574203A20426173655F31A3
:10182C00384632374B34325F546573745F534D54C2
:10183C00315F57696E646F7765645F73696E676C4F
:10184C00655F61735F467265716D657465725F3259
:0F185C003032315F31312E6D637070690D0A00CB
:10186B00205465737420534D5420636F6D707465F1
:10187B0075722032342062697473202872E9737593
:10188B006DE92064657320726567697374726573A3
:10189B0020656E20706167652033363429200D0A70
:0118AB00003C
:1018AC0020496E697420496E74657272757074206B
:0B18BC0055415254205258200D0A00E4
:1018C7002020436C6F636B20696E697469616C6576
:0B18D70020696E204B687A203D200045
:1018E20020506F77657220737570706C793A20336F
:0A18F2002E3620E02035560D0A00C6
:1018FC002049565420496E74657272757074206D4F
:08190C006F646520210D0A0043
:10191400205465737420706F696E746575722053FA
:0519240054203A2000F0
:10192900204D4355203A2031384632374B34320D59
:021939000A00A2
:10193B0020464F534320203A2036344D487A0D0A27
:01194B00009B
:10194C0030313233343536373839414243444546E9
:0C195C000D0A205265E775203A0D0A00C4
:0819680020467265713D20006C
:020000040030CA
:0A00000004092FB70B3E9F0F01000B
:00000001FF
